:020000040000FA
:10000000DFEF05F07080000C056ED8CF06F0E950E8
:10001000076EEA50086EE150096EE2500A6ED95040
:100020000B6EDA500C6EF350146EF450156EE050F7
:100030000D6E000100500F6E0150106E0250116ED7
:100040000350126E0450136E9DA02AEF00F09EB074
:100050007FEF05F0A0AA30EF00F0A1BA64EF05F041
:100060000F50006E1050016E1150026E1250036E50
:100070001350046E0D50E06E0D8E0750E96E08505F
:10008000EA6E0950E16E0A50E26E0B50D96E0C50C8
:10009000DA6E1450F36E1550F46E055006C0D8FF9A
:1000A0001000F76AB20FF66E000EF7220900F55045
:1000B000120005010904A1010901A100093009315B
:1000C0001581257F75089502810205091901290806
:1000D00015002501750195088102C0C0F76AEC0F73
:1000E000F66E000EF7220900F550120009022200F8
:1000F000010100C0320904000001030102000921CE
:1001000000010001222A000705810304000AF76AA2
:100110001E0FF66E010EF7220900F55012000900BD
:10012000F76A300FF66E010EF7220900F550120043
:100130001B00F76A420FF66E010EF7220900F55018
:1001400012001201100100000008610421000001EA
:1001500001020001F76A640FF66E010EF722090032
:10016000F550120000041800F76A780FF66E010EC1
:10017000F7220900F55012000403090414035A0081
:10018000650072006F002D0053006F006600740060
:1001900032035A00650072006F002D0053006F009B
:1001A0006600740020004E0045005300200043000C
:1001B0006F006E00740072006F006C006C006500D0
:1001C0007200F2CF0EF0F29EF76ADC0FF66E010EAF
:1001D000F7220900F5500EBEF28E12000D0A0D0A2C
:1001E000555342204E455320436F6E74726F6C6CB2
:1001F00065720D0A0000F2CF0EF0F29EF76A100F42
:10020000F66E020EF7220900F5500EBEF28E1200B5
:10021000627920447265772048616C6C202864689C
:10022000616C6C407A65726F2D736F66742E636FAC
:100230006D0D0A0D0A00F2CF0EF0F29EF76A500F14
:10024000F66E020EF7220900F5500EBEF28E120075
:1002500057616974696E6720666F7220656E756D8F
:1002600065726174696F6E00F2CF0EF0F29EF76AEC
:10027000820FF66E020EF7220900F5500EBEF28EC6
:1002800012000D0A0D0A456E756D65726174656424
:100290000D0A0000F2CF0EF0F29EF76AAE0FF66E76
:1002A000020EF7220900F5500EBEF28E12000D0A62
:1002B0000D0A44657669636520556E2D636F6E6621
:1002C0006967757265642E0D0A003E6A3E5213E13D
:1002D000036A3E502A0FE96E000E0320EA6EEF6AB1
:1002E000036A3E50290FE96E000E0320EA6E010EEC
:1002F000EF6E3E2AEBD7206A226A010E236E216A36
:10030000000CE3DF6896689668966896880E04018C
:10031000006F050E036F026B080E016F046F050E70
:10032000076F080E066F6E6A68906D98160E706EF5
:10033000716A726A390E696E010E506E000167EFC4
:1003400005F0689469946D92689869886DEF05F07E
:1003500068986D826894698470EF05F0020E4E6EA5
:10036000040E4F6E4A50080DF3504E26000E4F22D9
:10037000010E4E24016E000E4F20036E01C0E9FFF6
:1003800003C0EAFFEFCF54F04EC0E9FF4FC0EAFFD1
:10039000EFCF55F054C052F055C051F04E50D8B484
:1003A0004F064E064EC0E9FF4FC0EAFFEFCF53F0B5
:1003B0004D50535C02E253C04DF04EC0E9FF4FC0B8
:1003C000EAFF080EEF6E4E50D8B44F064E06536A41
:1003D0004D50535C14E251C0E9FF52C0EAFFEFCF29
:1003E00056F04CC0EAFF4BC0E9FF56C0EFFF4B2A66
:1003F000D8B44C2A512AD8B4522A532AE9D72552C4
:1004000003E025C053F00CD04EC0E9FF4FC0EAFF17
:10041000EFCF53F0C00E5316400E531A880E5312EE
:100420004EC0E9FF4FC0EAFF53C0EFFF4DC001F0DF
:10043000000C040E4C6E4D6E4650080DF3504C26C9
:10044000000E4D224DC003F04CC0E9FF4DC0EAFF45
:10045000EFCF51F051BE62D0020E4C26000E4D225D
:10046000010E4C24016E000E4D20036E01C0E9FF09
:1004700003C0EAFFEFCF51F04CC0E9FF4DC0EAFFE7
:10048000EFCF52F051C04FF052C04EF04B6A49507E
:100490004B5C14E247C0E9FF48C0EAFFEFCF53F0DE
:1004A0004FC0EAFF4EC0E9FF53C0EFFF4E2AD8B459
:1004B0004F2A472AD8B4482A4B2AE9D74C50D8B4F7
:1004C0004D064C064CC0E9FF4DC0EAFF49C0EFFFA6
:1004D0004C50D8B44D064C064A2C0DD04CC0E9FF08
:1004E0004DC0EAFFEFCF4BF0C00E4B16400E4B1A3B
:1004F000880E4B120AD04A5203E1C80E4B6E05D04B
:100500004A50020802E1880E4B6E4CC0E9FF4DC014
:10051000EAFF4BC0EFFF010E016E02D0000E016E2C
:10052000000C466A486A180E476E42C049F04A6A93
:1005300080DF0150000C466A486A476A496A4A6A85
:1005400078DF000C446A285232E0445007082FE359
:100550002450FC0F1FE2040FE7EF02F0036A27505C
:10056000BDDD016E01C045F015D0036A275099DD4D
:10057000016E01C045F00ED0036A2750F5DD016E13
:1005800001C045F007D0036A2750D3DD016E01C0DA
:1005900045F000D0272A28064450442A036A180F41
:1005A000E96E000E0320EA6E45C0EFFFCCD728525B
:1005B00004E14450080801E0216A466A486A180EBE
:1005C000476E44C049F043C04AF033DF000CE824D2
:1005D000E90FF66E050EF76ED8B0F72A0A00F5504F
:1005E000FA6E0800F550F96E5C056A057805860517
:1005F000276A246A1B50010A0DE0030A10E0060A6C
:1006000011E0010A1CE0060A27E0220A34E0030A8E
:100610003BE03FD0120E286E030E246E3DD0220E1A
:10062000286E3AD0036A1A5072DD016E01C027F0BD
:10063000036A275053DD016E01C028F02DD0036AF4
:100640001A506EDD016E01C027F0036A275046DDA7
:10065000016E01C028F020D0020E246E036A1A50E9
:1006600079DD016E01C027F0036A27507DDD016E40
:1006700001C028F011D0120E276E036A27502EDD1C
:10068000016E01C028F008D0010E246E2A0E286EDB
:1006900003D0B8DC0CD000D01F5205E128501E5CFE
:1006A00002E21EC028F0010E216E436A4BDF000CEF
:1006B000710E436E0F0E446E506A425217E1020EE5
:1006C000506E0F0E446E710E436E44500F080DE3D2
:1006D00003E143507E0809E343C0E9FF44C0EAFF59
:1006E000EF6A432AD8B4442AF0D70DD0030E506ED7
:1006F000480E04010C6F100E0E6F050E0F6F120ED8
:10070000716E726A0001C3EF03F01950000A0DE028
:10071000010A12E0020A18E0060A1DE0030A21E0BD
:100720000E0A21E0010A25E030D023C018F0196A32
:10073000020E426EF6DE2BD01A2C04D0010E2316C8
:10074000FADE01D05FDC23D01A2C03D02382F3DE43
:1007500001D058DC1CD0020E216E1AC026F0EBDE50
:1007600016D046DF14D022C018F0010E426ED9DE3A
:100770000ED01A50010802E245DC06D01AC022F061
:100780001AC042F095D7D7DE02D03CDC00D001EF92
:1007900005F01950000A07E00A0A0BE0010A1CE004
:1007A0000D0A29E02AD0186A196A020E426EB9DED3
:1007B00026D022520FE01C520DE1036A1C502A0F72
:1007C000E96E000E0320EA6EEFCF18F0010E426EC4
:1007D000A8DE01D017DC13D022520BE0036A1C50B4
:1007E0002A0FE96E000E0320EA6E1AC0EFFFA3DEA7
:1007F00001D008DC04D0FCDE02D004DC00D001EF24
:1008000005F042500F0B700F436E0F0E446ED8B0C0
:10081000442A43C0E9FF44C0EAFFEF9047EF04F0E9
:1008200042500F0B700F436E0F0E446ED8B0442A27
:1008300043C0E9FF44C0EAFFEF8050EF04F04250AC
:100840000F0B700F436E0F0E446ED8B0442A44C095
:1008500003F043C0E9FF44C0EAFFEFCF45F0000ECC
:1008600045B0010E016E57EF04F01C507F0B0E08CF
:1008700003E202EC00F024D01950010A05E0020A5C
:1008800008E0030A0FE01BD01CC042F0BAD753DEC9
:1008900017D01C500F0B000A04E01CC042F0C0D758
:1008A0004ADE0ED0186A196A1CC042F0C8D701523D
:1008B00002E0010E186E020E426E33DE01D000D04F
:1008C00001EF05F0485000D0526A516A00D04950FB
:1008D0004A1009E049C0E9FF4AC0EAFF52C0ECFFF4
:1008E000ED5251C0EFFF4B504C1009E04BC0E9FFF7
:1008F0004CC0EAFF54C0ECFFED5253C0EFFF4D5027
:100900004E1006E04DC0E9FF4EC0EAFF4FC0EFFFBA
:1009100096EF04F042C048F04A6A430E496E4C6AB2
:10092000450E4B6E4E6A470E4D6ECCD74350441069
:100930002FE043C001F044C003F043C048F044C07E
:1009400049F042C04AF046C04CF045C04BF047C0A9
:100950004DF004DD49C0EAFF48C0E9FF01503F0BFC
:10096000006ED89000360036030EEF140010EF6EC4
:1009700043C0E9FF44C0EAFFEFA005D043C0E9FF50
:1009800044C0EAFFEF8243C0E9FF44C0EAFFEF80C2
:10099000000C1950030A05E0080A10E0020A19E0E9
:1009A0001BD0036A1C50290FE96E000E0320EA6E6B
:1009B000EFCF18F0010E426EB4DD11D0036A1C5067
:1009C000290FE96E000E0320EA6E1AC0EFFFB3DDB7
:1009D00006D0426A9FDF03D002EC00F000D001EFA6
:1009E00005F0216A18507F0B000A07E0010A06E0B3
:1009F000030A05E0230A04E004D087D6CAD635D717
:100A0000C8D752EF05F0446A43C06EFF435202E07C
:100A1000020E446E44C050F013EF05F0226A216AC2
:100A200026C043F0F0D721EF05F042520AE1212C15
:100A300004D0010E436E86DD04D02150020801E18E
:100A4000EDD75AEF05F068A63DD06CCF3FF0040E0D
:100A5000416E406A68963F504026000E412240C0D9
:100A6000E9FF41C0EAFFEFCF3EF03C0E3E163F509B
:100A7000180B006E00303F6E3F323F321F0E3F16A4
:100A80003E50340811E1880E256E4A6A4C6A180EF1
:100A90004B6E080E4D6E62DC256A080E0401046F71
:100AA00000019FD76D980DD03E50240804E13FC04F
:100AB00042F0BBD706D03E50040803E13FC042F0ED
:100AC00029DFC1D773EF05F068A001D01AD468A25E
:100AD00001D0689268A401D034D468A801D038D479
:100AE00068A601D0B0D768BC689C68BA689A68529A
:100AF000EBE10A01F09BA19A000130EF00F0FE0E3D
:100B0000CF6E0C0ECE6E2C5205E1898492948992A0
:100B100092922CD02C2C0BD0899492942D6A928096
:100B200080A002D0D89001D0D8802D321FD02C5078
:100B30000F080EE1928080A002D0D89001D0D8801A
:100B40002D32899292922DC02BF0FF0E2C6E0ED07A
:100B50002CA00AD0928080A002D0D89001D0D8805A
:100B60002D328992929202D0898292922C2A2C5014
:100B70000F0801E22C6A9E9030EF00F0506A010EDF
:100B8000696E6E6A080E6D6E140E6F6E176AF2BE95
:100B9000178EF29E65EC01F017BEF28EA08AC00E91
:100BA000F212FEEF05F0EA6A310EE96EEF5006E050
:100BB000520E006E002EFED7EF2EFAD7000CF86A08
:100BC000D09E0D8EEA6AE96AC150C00B0F09C16E52
:100BD000070EB46EB450A19CB8860C0EAF6E000E1A
:100BE000B06E260EAC6E900EAB6E256A286A2C6A2B
:100BF0002D6A010E926E850ECD6EC0D7D1809D807C
:100C0000C00EF212316A3150E1EC00F0312A006E70
:100C100000509EA8FED7AD6E180E315CF4E1316A2B
:100C20003150FBEC00F0312A006E00509EA8FED738
:100C3000AD6E250E315CF4E1316A31501BEC01F0F0
:100C4000312A006E00509EA8FED7AD6E170E315CA3
:100C5000F4E1030E326E2E0E9EA8FED7AD6E322E3C
:100C6000FAD78A9093908A92939222520BE10400D1
:100C70002E0E9EA8FED7AD6E93908A70FA0E316E3E
:100C800092DFF3D7316A315034EC01F0312A006E33
:100C900000509EA8FED7AD6E040E315CF4E1030E49
:100CA000326E2A0E9EA8FED7AD6E322EFAD7040EF3
:100CB000336E335034EC01F0332A006E00509EA89E
:100CC000FED7AD6E0E0E335CF4E1030E346E2A0EC9
:100CD0009EA8FED7AD6E342EFAD70D0E9EA8FED775
:100CE000AD6E0A0E9EA8FED7AD6E8A8093908A8262
:100CF0009392225239E004002E6A2F6A306A2BA0A8
:100D000001D030802BA201D030822BA401D03084BE
:100D10002BA601D030862BA803D03088810E2F6EF1
:100D20002BAA03D0308A7F0E2F6E2BAC03D0810EFE
:100D30002E6E308C2BAE03D07F0E2E6E308E176A47
:100D4000F2BE178EF29E010E466E486A2E0E476E58
:100D5000030E496E010E4A6E19EC02F017BEF28EB8
:100D60000A0E316E20DFC5D7316A31504AEC01F0EE
:100D7000312A006E00509EA8FED7AD6E1B0E315C6E
:060D8000F4E16FD703004F
:00000001FF
